:020000020000FC
:10000000FBC991C20000000025C000004FC10000E4
:10001000000052C1000000000000000002030406BE
:10002000080C101820304060800002030406080C01
:10003000101820304080FF000406080C10182030F3
:10004000406080A0C0000D0D0403060D050D0603E1
:10005000030202004FB662FD1EC070FF1AC165FDAB
:10006000FAC00994C0919700C395C0939700C5E06A
:10007000C519B8F3D0919700CD1B98F3C8E7089441
:1000800083FDC795C4BDC52DCC2321F4C0E083FDFD
:10009000C0E8C4BD09C171FF03C0909A949A959AB3
:1000A000C52D089483FDC795C4BDC09399006B7F8F
:1000B000C52DCF3F09F443C0C0919800C395C093AC
:1000C000980070FF37C082FD05C0909A949A959A67
:1000D0004FBE18957860C091A000CC2391F0C091DC
:1000E0009800CA95D091A000CD1B58F0777FC091A1
:1000F0009800D0919F00CD1B08F41CC0209298005E
:1001000019C0909A949A959AC5E0CA95F1F7C09152
:100110007500CA95C2FD09C0C1FD05C095FF979A3B
:1001200095FD919A0EC0939A0CC095FF919A95FDFA
:10013000979A07C0909A949A959A4FBE18952092D4
:1001400099004FBE1895A5C0552021F095FF9098B5
:1001500095FD9598949A9DC0552009F0949895FF27
:10016000959A95FD909A95C0552021F095FF959808
:1001700095FD909895FF909A95FD959A8AC095FF68
:10018000919895FD979895FF979895FD9198C5E062
:10019000CA95F1F7552021F095FF909895FD959817
:1001A000949A77C095FF919895FD97989398C5E09C
:1001B000CA95F1F7552021F095FF909895FD9598F7
:1001C000949A67C0939895FF919895FD9798C5E08C
:1001D000CA95F1F7552009F0949895FF959A95FDE9
:1001E000909A57C0939895FF979895FD9198C5E080
:1001F000CA95F1F7552009F0949895FF959A95FDC9
:10020000909A47C095FF979895FD91989398C5E06F
:10021000CA95F1F7552021F095FF959895FD909896
:1002200095FF909A95FD959A34C095FF979895FD06
:10023000919895FF919895FD9798C5E0CA95F1F72B
:10024000552021F095FF959895FD909895FF909AEF
:1002500095FD959A1EC082FF1CC0C0917500C2FD1D
:100260000BC0C1FD11C095FF919895FD979895FF22
:10027000979895FD91980DC0C1FDF5CF95FF919888
:1002800095FD9798939805C0939895FF979895FD3D
:100290009198C52DC095089483FDC795C4BDC093A2
:1002A00099002092970064604FBE18954FB6C0E148
:1002B000C8BF6E7F4FBE18953FB68F7EABB7A07498
:1002C000A2118061A0E0ABBFA9B7AE7FA9BF7894AF
:1002D000A0916600AA2349F0A92FAF7151F1A09116
:1002E0006600AA95A093660024C040E050E0A0B349
:1002F00096FFA095A2FD4FEF96FDA3E096FFA2E02A
:10030000A5BFAA27A064AABF8D7FA0B396FFA09522
:10031000A2FD5FEF451749F7A0E461FDA0936600D9
:10032000A92FAF7119F0A0E4A093660040938D004F
:100330008160A0916700AA2331F0A0916700AA957F
:10034000A093670007C0A92FAF7121F08061AA2791
:10035000A064AABF80FF30C0A0918D004A2F8E7F7D
:10036000A92FAF7109F000C04093610071FF08C070
:10037000A091610050919200A51710F05093610078
:100380004091AE004430C1F4A091610040916300FF
:10039000A41B70F04091CF00A40B50F0A09163001B
:1003A000A40FA093630040F4AFEFA093630004C0D8
:1003B000A0916100A0936300A52DA03408F06860AF
:1003C000A0916000A395A093600051F0F894A9B7A4
:1003D000A160A9BF84FF02C0A0E4ABBF3FBE1895D7
:1003E00042E050916600552331F0A92FAF7119F406
:1003F0005A9550936600A0918D00A13018F020927C
:1004000090000DC02092910020929A00A09190003F
:10041000AF5FA093900018F0AFEFA0939000B09062
:1004200061005091AE00523049F466FF91F0A2E3B2
:10043000BA1678F0A0917F00A0936100533049F480
:1004400066FF39F0A2E3BA1620F0A091BA00A0939B
:100450006100509162005B1521F010F05A9501C0C7
:100460005395509362004A95D1F650919A00539556
:1004700009F45A9550939A00A0919B00AA95A093D5
:100480009B0009F046C0A1E0A0939B0045E0A0912D
:100490009C005A17F0F1A0919D005A1728F441E0F2
:1004A000A3E0A0939B0007C0A0919E005A1718F4E8
:1004B00041E040939B00D0909300C0906300DC1417
:1004C000A8F0A091AE00A430D9F066FD0FC0C09294
:1004D0009300539519F0A0919C00A0939A00A1E07D
:1004E000A0939B00ACE3A093620013C0A091930083
:1004F000A40F20F45FEF5093930002C0A0939300E9
:10050000A0919300AF3F29F4AFEFA0939100A09387
:100510009A00F894A9B7A160A9BF84FF02C0A0E423
:10052000ABBF3FBE18953FB64CB55DB58F7EABB740
:10053000A074A2118061A0E0ABBFA9B7AE7FA9BF34
:10054000789481FD26C096FDA2E096FFA3E0A5BFAA
:100550008260A0B396FFA095A2FF05C040936400FF
:1005600050936500FDC096FDA3E096FFA2E0A5BFF5
:10057000AA27A064AABF8D7FA92FAF7109F4E1C09B
:1005800040E0A0B396FFA095A2FDDBC040938D0094
:10059000CEC096FDA3E096FFA2E0A5BF8D7F61FFD0
:1005A0006BC096FDA2E096FFA3E0A5BFAA27A064BA
:1005B000AABF82604093880050938900A090860073
:1005C0004A19B09087005B09BB24A2E0EA2EA22C56
:1005D000483CA0E05A0730F4A0E1BA2EE22CAAE091
:1005E000AA2E27C04836A1E05A0730F4A8E0BA2E58
:1005F000E22CAFE0AA2E1DC0403DA2E05A0730F425
:10060000A4E0BA2EE22CAEE1AA2E13C0403AA5E037
:100610005A0730F4A2E0BA2EE22CACE3AA2E09C0AD
:100620004839A8E05A0728F4A1E0BA2EE22CA8E73E
:10063000AA2EC42EA0918A00CA1AD52EA0918B0092
:10064000DA0ADD202AF4AFEFC094D094CA1ADA0A8D
:1006500020928C00CA14DE0418F4A1E0A0938C0050
:1006600040938A0050938B004091880050918900FC
:100670004093860050938700A09164004A1BA0918C
:1006800065005A0B94FD46C093FD44C092FD40C0E6
:100690005695479591FD3CC05695479590FD38C0BD
:1006A000D52EC42ED694C79461FD0CC0AC2DAC5190
:1006B000AD2DA24008F045C0DD2021F4AC2DA85C92
:1006C00008F43FC0A0E0EA2E97FD02C0E090C2000F
:1006D000AAEFEA0EF22CF21CCE18DF084FB74170D9
:1006E000442319F040E050E015C0AFEFCA16D20421
:1006F00018F04FEF50E00EC0F090A700CF9C412DB6
:10070000000C441F50E008F012C04FEF50E00FC043
:100710005695479594FF07C0552309F04FEFA42F36
:10072000A6954A0F521D4F3F520508F04FEF4093D8
:100730008D00816061FF05C0AFE1A095A923AB29C1
:100740009A2FA0E4A0936600A92FAF7119F4AAE034
:10075000A093660061FD04C0A92FAF7109F08F7EE0
:10076000A0E2A0936700A92FAF7119F4AAE0A093AB
:100770006700F894A9B7A160A9BF84FF02C0A0E4F4
:10078000ABBF3FBE189511E00AC013E008C01AE0E5
:1007900006C01EE104C014E602C018EC00C005E16A
:1007A000BB27BA95F1F70A95D9F71A95C1F70895BD
:1007B0002AE338E709C020E33CE806C02AE234EB2C
:1007C00003C025E238EC00C0652CB1E05B2E12E0DE
:1007D00095FD9F7D95FF9062BB279398BA95F1F7A1
:1007E000552009F09498BA95F1F7949ABA95F1F7D3
:1007F000939ABA95F1F7552021F095FF909895FDC1
:100800009598B091A800BA95F1F795FF909A95FD4B
:10081000959AB7E8BA95F1F71A95D1F6022FB22F4B
:10082000BA95F1F70A95D9F73A9571F69398562C3F
:100830000895221B39E0001F3A9509F40895221FFC
:10084000211B18F4210F8894F6CF0894F4CF622C62
:10085000722CB0E08894B395221F331FE0F73795D0
:1008600027958894912E802E020B130B10F4192DCE
:10087000082D10F4889401C00894661C771CBA9562
:1008800071F7172D062D0895322D11232AF43A956C
:1008900000951095031B130BF894029F712C002DEB
:1008A000129F912C802C7894780C172D921C292D56
:1008B000B4E06B2E2695179507956A94D9F73323E4
:1008C00021F000951095031B130B08950091AE00C5
:1008D000043009F474C0B0918D00B95198F0B72F6D
:1008E000B67081F466FD2BC005E09090C000B92D74
:1008F000BA9521F00AE0BA9509F002E1B0917400CE
:10090000B01BE0F066FF0AC0B0919500B093930071
:10091000BFEFB0939A00B1E0B0939B00B09161003B
:10092000B0936300209277002092780020927900A3
:1009300020927A0020927B006F7B41C0606490908F
:10094000C000B92DBA9579F4B0916200B095BB1F83
:10095000BB1F1B2FB7950B2FB12FB170B3951B2F5A
:10096000B02FBE7F25C0B92DBA95BA9581F4B0914C
:100970006200B095BB1FBB1FBB1F1B2FB7950B2F72
:10098000B12FB370B3951B2FB02FBC7F14C0B091A3
:100990006200B095BB1FBB1FBB1FBB1F1B2FB795B2
:1009A0000B2FB12FB770B395B3951B2FB02FB87F16
:1009B000B0540B2F1209009377001093780008951C
:1009C00066FF21C010917400169500917300079581
:1009D000B0917700B01B0B2FB0917800B10B1B2F9B
:1009E00028F40038BFEF1B0740F009C00F3712058D
:1009F00008F405C00FE710E002C000E81FEF009305
:100A00007C0010937D00089566FF39C000917C0042
:100A1000B09179000B0F10917D00B0917A001B1FEF
:100A200020E030917D0033230AF42A95B0917B00B9
:100A30002B1F1AF4203F40F00AC02F3008F407C0E3
:100A40000FEF1FEF2FE003C000E010E020EF309128
:100A50006300B09192003B1718F4332331F009C0C2
:100A6000B0917D00BB235AF004C0B0917D00BB2340
:100A700032F40093790010937A0020937B0008955C
:100A800066FF2FC02091CD0000917C00000F1091D7
:100A90007D00111FF9DE11232AF40038BFEF1B0778
:100AA00040F009C00F37120508F405C00FE710E049
:100AB00002C000E81FEF002352F0B0916200B01BAB
:100AC0000B2F18F0013008F00AC001E008C00095B3
:100AD0000F5FB09162000B0F08F001C00FEF0093A1
:100AE0007E00089566FF2DC02091CE0000917A000F
:100AF00010917B00C9DE11232AF40130BFEF1B07E0
:100B000040F009C00F3F120508F405C00FEF10E0D8
:100B100002C001E01FEF112352F0B0917E00B01B24
:100B20000B2F18F0013008F00AC000E008C0009553
:100B30000F5FB0917E000B0F08F001C00FEF009324
:100B4000630008950FEF677FB72FB670E9F4686010
:100B5000B0917400B83008F0677FB0917400A1F0D4
:100B60000FEF1091740065DEF894B09170000B9F48
:100B7000112D002D7894112309F00FEFB0919500FD
:100B80000B1710F4009195000093940008950AD378
:100B900074FFB7E074FDB7E0B068B064B7B9B6B140
:100BA000B068B064B6B9EFDD74FFB7E074FDB7E0CC
:100BB000B068B064B7B9B6B1B068B064B6B9B6B130
:100BC000B6FDFDCF04B115B1B6B1BF77B6B923D329
:100BD00024E32093A30030E03093A400732E769496
:100BE000622E6694620E731E262D372D0217130790
:100BF00078F08090A300B4E3B80DB093A300809088
:100C0000A400B0E0B81DB093A400260D371DEECFB0
:100C10008090A3009090A4001091A40016950091DC
:100C2000A300079516950795B091A300B00FB09358
:100C3000A100B091A400B11FB093A20023E01695CB
:100C400007952A95E1F72091AF002A9529F4209283
:100C5000A3002092A4000AC02A9521F0800E911EC4
:100C60002A95E1F78092A3009092A4000895209124
:100C7000AF00B6B1B6FDFBCF04B115B1B6B1BF77C9
:100C8000B6B9B091A500B395B093A500B83060F1A6
:100C90002092A500B091CC00BB2321F1112329F0B3
:100CA000B091A600BF3F61F009C0B091A6000B173C
:100CB00039F020F4BB2321F0BA9502C0B395E1F3DB
:100CC00000919200B093A600B03050F400ECB03028
:100CD00038F400E8B03020F400E4B03008F400E06C
:100CE000009392007F7E0895213099F00F3FB3E08A
:100CF0001B0778F4B091A3000B17B091A4001B0759
:100D000040F4B0919200BB2359F0BA95B093920091
:100D100007C0B0919200BF3F19F0B395B093920015
:100D200000919200B0916300B01B10F40091630039
:100D3000B09193000B1750F000919300B091930085
:100D4000BF3F21F0B0919300B0939200502EB0912C
:100D5000A500B73009F47061089502E3F894B091EA
:100D6000D0000B9F012D000C001F7894B0919200D1
:100D70000B1710F000919200009361000093630044
:100D8000502E00939500089520927300B8E0B09320
:100D9000740008952091800030918100F8940CB582
:100DA0001DB5200F311F3BBD2ABD6160B0E1B8BF4A
:100DB000789420917100309172000093710010932B
:100DC0007200021B130B2091730030917400622E8D
:100DD000732EB4E08B2EB2E09B2EB0917400B43031
:100DE00010F08A949A94B83010F08A949A94769479
:100DF00067948A94E1F726193709992021F016950E
:100E000007959A94E1F7200F311F209373003093D8
:100E1000740008F00895BFEFB0937300B0937400AE
:100E200008952091820030918300F8940CB51DB58F
:100E3000020F131F1BBD0ABD6160B0E1B8BF7894FB
:100E4000089560FDFECFEDDF0895B091BE000091E2
:100E50006E00023808F0B395003A08F0B395B6304A
:100E600008F0B5E09B2EBCE08B2EB0917400B3303F
:100E700030F48394839482FF02C083948394B230CD
:100E800030F48394839482FF02C08394839471FF2F
:100E900003C0B3E09B2E822C10917400009173006C
:100EA00024E0169507952A95E1F70819120928F00C
:100EB000B02FB250B12FB20910F402E010E0312F80
:100EC000202F712E602E76946794B92DB330E9F0FF
:100ED000B0FD05C0060D171D262D372D06C0000FCD
:100EE000111F0250120922E030E0B92DB33068F032
:100EF000209384003093850000938000109381003C
:100F00006092820070928300089500938400109391
:100F1000850020938000309381006092820070925F
:100F20008300089560FDFECF20918200220F309152
:100F30008300331FB72FB67021F0209173003091DA
:100F40007400F8940CB51DB5020F131F1BBD0ABD2C
:100F50006160B0E1B8BF7894089560612092760036
:100F600020E004C060612092760020E2B72FB670C6
:100F700009F06F7E789460FD05C0B0917600BB23C8
:100F800009F0089501E063FF0AC0B0917400B33026
:100F900008F002E0B0917400B63008F003E071FF91
:100FA00001C006E060FD06C0B0917600BB2311F0E1
:100FB000789408951AE083FF1AE078940000000006
:100FC000F89462FD03C014E183FF14E171FF01C0D6
:100FD00018E7B4B530919900B31BB10B18F3B09179
:100FE0007600B395B0937600B5E03B2F6B2E722C54
:100FF000B8B1B072B21709F073943A95C9F7739407
:10100000761488F464FFB2CF6F7E3CB56DB47090F7
:10101000730080907400370D681C6BBC3ABD616032
:10102000B0E1B8BFA3CF64FDA1CF0A9509F0BACF54
:101030007894089571FF0AC0B0916D00B395B09394
:101040006D0060FD0CC020926D0009C060FD07C0FE
:1010500064FD05C067FD03C0BF91BF9173C40895CF
:101060002091840030918500F8940CB51DB5020FD5
:10107000131F1BBD0ABD6160B0E1B8BF789408952D
:10108000EFDF00E063FF03C064FF01C001E0F894FC
:1010900010916E00B7E01B9F212D102D7894200F2A
:1010A00026951795269517952695179510936E00FA
:1010B000183718F4B8E7B0936E0000916E00B09145
:1010C0006F000B1720F06062909A949A959A60FDD9
:1010D000FECF0895F89491989398979882FF07C04F
:1010E000E2E0F1E073FF03C0B5E0BA95F1F795FFD8
:1010F000919A95FD979AB2E0B093750089C0F894E3
:1011000095FF959A95FD909A82FF0DC0E2EFF0E071
:1011100073FF0BC0939895FF979895FD9198B5E054
:10112000BA95F1F702C0ECEAF0E062FF03C0552087
:1011300009F09498B3E0B09375006AC0F894919860
:101140009398979882FF07C0E2EEF0E073FF03C028
:10115000B5E0BA95F1F795FF979A95FD919AB4E0AD
:10116000B093750055C0F894949A82FF0DC0E2EDDB
:10117000F0E073FF0BC095FF919895FD97989398B9
:10118000B5E0BA95F1F702C0E4EAF0E062FF06C00C
:10119000552021F095FF909895FD9598B5E0B09376
:1011A000750036C0F89491989398979882FF07C07D
:1011B000EFEBF0E073FF03C0B5E0BA95F1F7939A57
:1011C000B6E0B093750024C0F89495FF909A95FD11
:1011D000959A82FF10C0E5E1F1E073FF0EC095FF24
:1011E000919895FD979895FF979895FD9198B5E002
:1011F000BA95F1F702C0E4EBF0E062FF06C05520BB
:1012000021F095FF959895FD9098B1E0B093750009
:101210006F7D7894089523EA30E0F901909A949ACA
:10122000959A9198939897986B7F0895ACEAB0E05F
:1012300007E00D9307E00D9301E00D9304E00D939B
:101240000FEF0D930D9309E00D9302E00D9301E074
:101250000D9301E00D93A8EBB0E001E00D9300E0E9
:101260000D9304EB0D930FEF0D930D930D9303E08E
:101270000D9301E00D9301E00D930FEF0D9305E247
:101280000D9300ED0D9308E70D9308EC0D9304E02A
:101290000D930DE00D9301E00D9300E00D930AE72F
:1012A0000D930AE00D9301E00D9308952091BF0086
:1012B00009E011E0223011F405E011E0233011F4CF
:1012C00005E012E0243011F405E013E0253011F4BC
:1012D00009E017E0263011F400E010E000939F00D1
:1012E0001093A0002091B3008B7F233009F4846019
:1012F000777F233009F47860B091B4009F7DB1FD11
:1013000090629F7BB091B500B1FD9064B22FB23076
:1013100011F0886001C0877F0895ECE1F0E0009152
:10132000AC000A95E00FF21DB491B093CD0000918E
:10133000AD000A95E00FF21DB491B093CE006BDFC3
:101340000895EAE2F0E00091C7000A95E00FF21D6F
:10135000B491B093CF005FDF0895E8E3F0E000912F
:10136000B2000A95E00FF21DB491B093D00053DFA4
:1013700008950091CB00002309F40395013108F092
:1013800001E1B02FB00FB00FB0939C001B2FB10F35
:10139000B10FB00FB0939D00B10FB00FB00FB0936D
:1013A0009E000895B091C8000FEF1CE0B23011F418
:1013B00000EA1AE0B33011F402E815E000936F0080
:1013C00010937000089508952091C2003091C300D9
:1013D00097FF02C020E03FEFB32FB21B6B2EB25835
:1013E00010F4B2E86B2E00E00395609EB12DB0586A
:1013F000D8F30093A7000895F894E3E0F0E0B9E093
:10140000B7BFB491B078C1F3F894A895B1B5B861FD
:10141000B1BDB0E0B1BDB4E0BEBFBFE5BDBFFBDE56
:10142000B4E0B8BBB4E1B7BBB0E0B5BBB0E0B4BBAF
:10143000B1E3B2BBBBEBB1BB2224A0E0B0E02D9284
:10144000AA31E9F7A0E6B0E00FEF2D920A95E9F78F
:10145000EDDE9DD22BDF61DF74DF7FDF8ADFA2DF6D
:10146000B2DFB2DF0091C4000093A800D4DEB2E086
:10147000B3BFB2E0BEBDB2E0B5BDF8948ED998D985
:1014800088D999D986D99AD984D918D386D985D9B2
:1014900082D9B1E5B8BFB9BFB0B7B860B0BFB6B117
:1014A000B460B6B970D9789472DBB0E4BBBFBB2727
:1014B000B064BABF8D7F71D9B1E0B093690062604A
:1014C00025E0B0918C00BB2309F425E05ED9B091F2
:1014D0008D00B230A8F3B92FBF7100918F00009337
:1014E0008E00B0938F00B01759F72A9551F76D7F92
:1014F00096FDB3E096FFB2E0B5BFBB27B064BABFBC
:101500008D7F49D942D902E0B92FBF7109F400E0BB
:10151000B0918D00B017B0F3F8944AD949D948D9A1
:1015200078943BD920927F0030D9B091B800B13087
:1015300008F46CC0B0916900B13008F467C0B92FED
:10154000BF71C1F0B0918D00BF3F08F45FC0F89447
:1015500038D9789420D9B0918D00B130C0F7F89483
:1015600027D915D925D9789416D9B0918D00BF3FC8
:10157000B0F3D6C2B8E09B2E9068F89425DF78943B
:101580000AD9F8949F7720DF80908D00B0918D006C
:10159000BF37789408F442C0F6D8F89412D97894FA
:1015A0009A9451F7B82DB550B093C300F6D8F8947B
:1015B0001BD289D27894BAE09B2E9068F89404DF0D
:1015C0007894E9D8F8949F77FFDE80908D00B091F1
:1015D0008D00BF37789478F7D6D8F894E9D8D7D863
:1015E000E7D878949A9449F7B82DBB5FB093C200BE
:1015F000D4D8F894F9D176D27894CDD8F894E4DEA2
:101600007894B0918D00BF3FC0F38AC200918D00E5
:10161000B0917F000B1710F000937F00BCD801E061
:10162000B091B400B35009F405E0B0918D00B0174B
:1016300008F07ACFF894C5D8C4D8C3D87894ADD878
:101640002092690020926A0020926B00B0916A009B
:10165000B395B0936A00BF3F69F5B0916B00B39545
:10166000B0936B00B091C60009E1BA9559F002E35E
:10167000BA9541F00DE7BA9529F00AEFBA9511F045
:1016800020926B00B0916B00B017A0F0B0916B008E
:10169000BA95B0936B00B4EBB0936A00B091C500FB
:1016A000B093A800F8948DD87894B091C400B0930A
:1016B000A80071D86CD8B0916600BB2321F4B92F73
:1016C000BF7109F4FCCEB0918D00B63008F4BECFE6
:1016D00062D8B0916600BB2309F4F1CEF8949BDD8B
:1016E000209261002092620020926300522C789434
:1016F000B091B100B09396002092770020927800CC
:101700002092790020927A0020927B002092A500FE
:1017100060E070E020926E0037DBB8E0B093A50087
:10172000706131D874FFB7E074FDB7E0B068B064A1
:10173000B7B9B6B1B068B064B6B9B6B1B6FDFDCF51
:1017400004B115B1B6B1BF77B6B9112309F00FEFE7
:101750000093A6008CDAB8E0B093A5007061809089
:10176000B300B2E0B093B300A1DD8092B300F8946F
:10177000BFEFB0939200F1DAB0916100B0939200A4
:10178000B0939300B09394007894B1E0B09361006B
:10179000B09363005B2EB0939B00B0919100B09327
:1017A0009A007160726020926D00FCDC0DDDF2DA4F
:1017B000EBDA4BDB04C07ADD2092A5007F7E95FF3B
:1017C000B4E095FDB2E0B068B064B7B9CBDB32DC11
:1017D00047DC7CD855DC7EDCDDDA33DB36DBA2DBB4
:1017E000B3E0B068B064B7B9B8DB24DC39DCE8D862
:1017F000A9D946DC84DCCEDA24DB27DB93DB95FF3A
:10180000B2E095FDB4E0B068B064B7B9ABDB12DC10
:1018100027DCFAD835DC92DCBDDA13DB16DB82DBA1
:1018200095FFB4E095FDB2E0B068B064B7B995DB60
:1018300001DC16DC25D924DC96DCACDA02DB05DB26
:1018400071DBB3E0B068B064B7B98CDBF3DB08DC04
:1018500049D916DCA7DC9EDAF4DAF7DA63DB95FF08
:10186000B2E095FDB4E0B068B064B7B976DB74FF60
:10187000B7E074FDB7E0B068B064B7B9B6B1B068AE
:10188000B064B6B9D7DBECDBFBDB9EDC83DAD9DAFC
:10189000DCDAEDD947DB71FF20C067FD1EC0B091D7
:1018A0009500B0939200B0939300B0919100B093E3
:1018B0009A00B1E0B0939B0014E624E1B0916D0072
:1018C000B11728F07D7F746020936C0006C0B09142
:1018D0008D00B13008F073CF35C072FF10C067FDC6
:1018E0000EC0B0916C00BA9511F47B7F64CFB093B9
:1018F0006C00B0918D00B13008F061CF23C0B09181
:101900009000B13058F0B0919500B0939300B09131
:101910009100B0939A00B1E0B0939B00B091900019
:10192000BA3F80F4B92FBF7121F4B0916600BB2398
:1019300049F0B091740000EF67FF01C000E6B017F6
:1019400008F43DCFF89467DC8090B300B2E0B09328
:10195000B300ACDC8092B300209261002092620060
:1019600020926300522C209296007E7F78940BD7B1
:1019700052DCB92FBF7129F4B0916600BB2309F482
:101980009ECDB091B900B13008F0BCCD5BCEEDE09A
:10199000F0E023D0053A09F01BC0EEE0F0E01DD0E6
:1019A0000A3509F015C03AE0ACEAB0E0E3E0F0E057
:1019B00014D00D9331963A95D9F735E1A8EBB0E004
:1019C000EFE0F0E00AD00D9331963A95D9F702C0D6
:1019D0002DDC0AD0E4E2F0E00895E199FECFEEBB01
:1019E000FFBBE09A0DB308951ED03AE0ACEAB0E038
:1019F000E3E0F0E00D910FD031963A95D9F735E15B
:101A0000A8EBB0E0EFE0F0E00D9105D031963A950B
:101A1000D9F712D00895E199FECF0DBBEEBBFFBB05
:101A2000E29AE19A0895EDE0F0E00FEFF4DFEEE0E6
:101A3000F0E00FEFF0DF0895EDE0F0E005EAEBDF16
:101A4000EEE0F0E00AE5E7DF08953091A9000091AB
:101A5000AA00313011F40093AC00323011F400933D
:101A6000AD00333011F40093AE00343011F4009324
:101A7000C000353011F40093AF00363011F40093FC
:101A8000B200373011F40093BE00383011F40093E7
:101A9000C700393011F40093BF003A3011F40093BD
:101AA000B3003B3011F40093C8003C3011F40093B4
:101AB000B4003D3011F40093B500089525E06DD6D3
:101AC0002A95E9F7089574D676D678D67AD65FD671
:101AD0006FD671D673D675D65AD66AD66CD66ED6F0
:101AE00070D608956ED66AD666D662D650D669D6B6
:101AF00065D661D65DD64BD664D660D65CD658D650
:101B000008958090A9009090AA0052D651D650D640
:101B10003ED68A94D1F755D63AD69A94E1F70895ED
:101B2000F894D1DF7894CADFC9DFB1E0B093A9009F
:101B3000B1E0B093AA002092AB00F894E2DF789471
:101B4000B5E06B2E70908D0028D6B0918D007B167D
:101B5000C9F7B13018F0BF3F40F107C076DFF89405
:101B600043DFB1DFB8E0B1BDA9DF6A9459F7B091A6
:101B7000AB00B395B093AB00B33008F4DECF9EDF7B
:101B8000B091AA00B395B093AA00F894B091A900BF
:101B9000BA95E6E4F0E0EB0FF21D0491789403951A
:101BA000B091AA00B01708F4C6CF88DF87DFB091E4
:101BB000A900B395B093A900B091A900BE3008F474
:0E1BC000B7CF34DBF89410DFB8E0B1BD77DFAB
:00000001FF
